:020000040000FA
:100000000C9490000C94B8000C94B8000C94B800B8
:100010000C94B8000C94B8000C94B8000C94B80080
:100020000C94B8000C94B8000C94B8000C94B80070
:100030000C94B8000C94B8000C94B8000C94B80060
:100040000C94520A0C94B8000C94200A0C94FA09EF
:100050000C94B8000C94B8000C94B8000C94B80040
:100060000C94B8000C94B80008000000BE9224491B
:10007000123EABAAAA2ABECDCCCC4C3E00000080DA
:10008000BEABAAAAAA3E00000000BF000000803F4D
:100090000000000000084178D3BB4387D1133D190D
:1000A0000E3CC3BD4282AD2B3E68EC8276BED98F3A
:1000B000E1A93E4C80EFFFBE01C4FF7F3F0000007E
:1000C000000000000000240027002A0000000000BB
:1000D000250028002B000000000023002600290036
:1000E00004040404040404040202020202020303DE
:1000F00003030303010204081020408001020408E6
:100100001020010204081020000000080002010075
:100110000003040700000000000000009C0A780DA6
:1001200011241FBECFEFD8E0DEBFCDBF25E0A8E38E
:10013000B4E001C01D92A830B207E1F714E0A0E0DE
:10014000B1E0E8E4F5E202C005900D92A833B107F2
:10015000D9F710E0CFE8D0E004C02197FE010E945B
:100160009610CE38D107C9F70E94D70A0C9497127F
:100170000C940000AF92BF92CF92DF92EF92FF9269
:100180000F931F93CF93DF936C017B018B01040FBF
:10019000151FEB015E01AE18BF08C017D10759F05B
:1001A0006991D601ED91FC910190F081E02DC6019D
:1001B0000995892B79F7C501DF91CF911F910F9197
:1001C000FF90EF90DF90CF90BF90AF900895FC012B
:1001D000538D448D252F30E0842F90E0821B930BAC
:1001E000541710F0CF96089501970895FC01918D52
:1001F000828D981761F0A28DAE0FBF2FB11D5D9655
:100200008C91928D9F5F9F73928F90E008958FEFF6
:100210009FEF0895FC01918D828D981731F0828DAA
:10022000E80FF11D858D90E008958FEF9FEF089501
:10023000FC01918D228D892F90E0805C9F4F821B65
:1002400091098F739927089581E694E00E9418011F
:1002500021E0892B09F420E0822F089580E090E0CE
:10026000892B29F00E94240181110C94000008952B
:10027000FC01A48DA80FB92FB11DA35ABF4F2C911B
:10028000848D90E001968F739927848FA689B78912
:100290002C93A089B1898C91837080648C93938D09
:1002A000848D981306C00288F389E02D80818F7DAC
:1002B00080830895EF92FF920F931F93CF93DF9364
:1002C000EC0181E0888F9B8D8C8D98131AC0E88992
:1002D000F989808185FF15C09FB7F894EE89FF8961
:1002E0006083E889F98980818370806480839FBFFF
:1002F00081E090E0DF91CF911F910F91FF90EF90FF
:100300000895F62E0B8D10E00F5F1F4F0F7311270E
:10031000E02E8C8D8E110CC00FB607FCFACFE88949
:10032000F989808185FFF5CFCE010E943801F1CF98
:10033000EB8DEC0FFD2FF11DE35AFF4FF0829FB7BD
:10034000F8940B8FEA89FB8980818062CFCFCF93AD
:10035000DF93EC01888D8823B9F0AA89BB89E889ED
:10036000F9898C9185FD03C0808186FD0DC00FB693
:1003700007FCF7CF8C9185FFF2CF808185FFEDCF11
:10038000CE010E943801E9CFDF91CF9108958330EB
:1003900081F028F4813099F08230A9F008958730F7
:1003A000A9F08830C9F08430B1F4809180008F7D4D
:1003B00003C0809180008F7780938000089584B57A
:1003C0008F7784BD089584B58F7DFBCF8091B00079
:1003D0008F778093B00008958091B0008F7DF9CF22
:1003E000CF93DF93282F30E0F901E85FFE4F84912F
:1003F000F901EC50FF4FD491F901E052FF4FC49145
:10040000CC23A1F081110E94C701EC2FF0E0EE0F88
:10041000FF1FEA52FF4FA591B491EC91ED2381E0CB
:1004200090E009F480E0DF91CF91089580E090E0C2
:10043000FACF1F93CF93DF93282F30E0F901E85FC5
:10044000FE4F8491F901EC50FF4FD491F901E05235
:10045000FF4FC491CC23A9F0162F81110E94C70130
:10046000EC2FF0E0EE0FFF1FE453FF4FA591B49186
:100470008FB7F894EC91111108C0D095DE23DC936E
:100480008FBFDF91CF911F910895DE2BF8CFCF93CF
:10049000DF9390E0FC01EC50FF4F249180529F4F7E
:1004A000FC0184918823D1F090E0880F991FFC0112
:1004B000EE53FF4FA591B491FC01E453FF4FC5915A
:1004C000D49161110EC09FB7F8948C91E22FE09502
:1004D0008E238C932881E223E8839FBFDF91CF9105
:1004E00008958FB7F894EC91E22BEC938FBFF6CF81
:1004F0003FB7F8948091530490915404A09155040F
:10050000B091560426B5A89B05C02F3F19F001965F
:10051000A11DB11D3FBFBA2FA92F982F8827BC015D
:10052000CD01620F711D811D911D42E0660F771F85
:10053000881F991F4A95D1F708958F929F92AF9285
:10054000BF92CF92DF92EF92FF924B015C010E942B
:1005500078026B017C010E9478026C197D098E097A
:100560009F09683E734081059105A8F321E0821A36
:100570009108A108B10888EEC80E83E0D81EE11CDE
:10058000F11C81149104A104B10429F7FF90EF90AC
:10059000DF90CF90BF90AF909F908F9008952FB72E
:1005A000F89460914F04709150048091510490919F
:1005B00052042FBF0895FC0101900020E9F7319704
:1005C000AF01481B590BBC0181E694E00C94BA00C2
:1005D000009711F00C94DB0290E080E008958F9278
:1005E0009F92AF92BF920F931F93CF93DF93CDB79C
:1005F000DEB7A1970FB6F894DEBF0FBECDBF19A22C
:10060000423008F44AE08E010F5D1F4F842E912C7A
:10061000B12CA12CA50194010E947410E62FB90100
:10062000CA01EA30D4F4E05DD801EE938D01232BAA
:10063000242B252B79F7CD010E94E802A1960FB655
:10064000F894DEBF0FBECDBFDF91CF911F910F9108
:10065000BF90AF909F908F900895E95CE5CFCF92C7
:10066000DF92EF92FF9260E08CE00E94190264E654
:1006700070E080E090E00E949D028CE191E00E9499
:10068000E80261E08AE00E9419026CED75E080E00A
:1006900090E00E949D0260E08AE00E94190261E001
:1006A0008BE00E9419020E94CF026B017C01C09274
:1006B0005B04D0925C04E0925D04F0925E046AE018
:1006C00070E080E090E00E949D0284E00E94F001D2
:1006D0000197E1F46CED75E080E090E00E949D02EE
:1006E00060E08BE00E94190264E670E080E090E038
:1006F0000E949D028BE291E00E94E80261E08CE0A2
:10070000FF90EF90DF90CF900C9419020E94CF02DF
:100710006C197D098E099F0969397A438105910514
:1007200070F264E670E080E090E00E949D0286E353
:1007300091E00E94E80260E08BE00E94190281E0F3
:1007400090E09093600480935F04D8CFCF92DF92C3
:10075000EF92FF9260E08CE00E94190264E670E084
:1007600080E090E00E949D0288E591E00E94E8020E
:1007700061E08BE00E94190268EE73E080E090E097
:100780000E949D0260E08BE00E94190261E08AE015
:100790000E9419020E94CF026B017C01C0925B048F
:1007A000D0925C04E0925D04F0925E046AE070E036
:1007B00080E090E00E949D0283E00E94F00101979A
:1007C000E1F464E873E080E090E00E949D0260E064
:1007D0008AE00E94190264E670E080E090E00E94E6
:1007E0009D028DE291E00E94E80261E08CE0FF90C2
:1007F000EF90DF90CF900C9419020E94CF026C19F9
:100800007D098E099F0969397A438105910570F246
:1008100064E670E080E090E00E949D0285E691E051
:100820000E94E80260E08AE00E94190281E090E004
:100830009093600480935F04D8CF60E08CE00E94C6
:10084000190264E670E080E090E00E949D0285E875
:1008500091E00E94E80261E087E00E94190268EEE0
:1008600073E080E090E00E949D0260E087E00E94DB
:10087000190264E670E080E090E00E949D0282E947
:1008800091E00E94E80261E08CE00C941902CF92A2
:10089000DF92EF92FF9260E08CE00E94190264E622
:1008A00070E080E090E00E949D028BE991E00E9460
:1008B000E80261E089E00E9419020E94CF026B0108
:1008C0007C01C0925B04D0925C04E0925D04F092E3
:1008D0005E046AE070E080E090E00E949D0282E0A9
:1008E0000E94F0010197B1F460E089E00E941902D2
:1008F00064E670E080E090E00E949D0288EA91E06A
:100900000E94E80261E08CE0FF90EF90DF90CF90D2
:100910000C9419020E94CF026C197D098E099F095F
:1009200069397A4381059105A0F287EB91E00E9435
:10093000E80260E089E00E94190264E670E080E06D
:1009400090E00E949D0289ED91E00E94E80281E022
:1009500090E090934D0480934C0490934B048093CB
:100960004A04D0CFFC0180819181009711F00C9452
:1009700038110895FC0124813581232B39F421E0BD
:10098000FB018081882349F020E007C080819181AC
:100990000E94871221E0892BB9F7822F08950F93C7
:1009A0001F93CF93DF93EC0188819981009759F0D1
:1009B0002A813B812617370730F081E0DF91CF9104
:1009C0001F910F9108958B016F5F7F4F0E94C1119E
:1009D000009759F0998388831B830A832C813D817A
:1009E000232B59F7FC011082E8CF80E0E7CFEF928C
:1009F000FF920F931F93CF93DF93EC017B018A014A
:100A0000BA010E94CF0428813981811114C02115B7
:100A1000310519F0C9010E943811198218821D820E
:100A20001C821B821A82CE01DF91CF911F910F9100
:100A3000FF90EF9008951D830C83B701C9010E94B8
:100A40009012F1CFFB0101900020E9F73197AF013F
:100A5000461B570B0C94F704FF920F931F93CF93F1
:100A6000DF93EC01198218821B821A821D821C827C
:100A700050E040E062ED73E00E94F704009102054F
:100A80001091030501151105F9F00430110510F05E
:100A900004E010E0E091FE04F091FF04E00FF11F8C
:100AA000F08010826091FE047091FF046115710561
:100AB00091F0CE010E9422058091FE049091FF04E6
:100AC000080F191FF801F082CE01DF91CF911F911D
:100AD0000F91FF90089588819981009711F00E94ED
:100AE0003811198218821D821C821B821A82E4CF5F
:100AF0000F931F93CF93DF9300D0CDB7DEB781E67E
:100B000094E00E941801892BA1F16AE070E080E076
:100B100090E00E949D0281E694E00E941801181660
:100B200019066CF781E694E00E94F60089831A8228
:100B300000910205109103050F5F1F4FB8018EEF62
:100B400094E00E94CF048823D1F22091FE043091DA
:100B5000FF048091020590910305BE016F5F7F4FF6
:100B6000820F931F0E9490121093030500930205B9
:100B7000C6CF0F900F90DF91CF911F910F910895E5
:100B80004F925F926F927F928F929F92AF92BF929D
:100B9000CF92DF92EF92FF921F93CF93DF9300D01B
:100BA00000D0CDB7DEB760E08CE00E94190261E0B2
:100BB0008DE00E9419020E94CF0260935B04709343
:100BC0005C0480935D0490935E046093440470938E
:100BD0004504809346049093470464E670E080E007
:100BE00090E00E949D0289EE91E00E94E80264E696
:100BF00070E080E090E00E949D02C0900001D090E3
:100C000001010D2C000CEE08FF084AE0C701B601F7
:100C1000F7FE0DC06DE281E694E00E945A0166275E
:100C20007727CB016C197D098E099F094AE00E9444
:100C3000EF0264E670E080E090E00E949D02109276
:100C4000400410924104109242041092430480E048
:100C500090E0A0E2B1EC80933C0490933D04A0931B
:100C60003E04B0933F0480E090E0A8ECB2EC8093A7
:100C7000380490933904A0933A04B0933B0417E4EA
:100C800088EE482E83E0582E612C712C10937C0046
:100C900080917A00806480937A0080917A0086FD4A
:100CA000FCCF8091780060917900762F682F072E15
:100CB000000C880B990B0E94830D9B01AC0160E036
:100CC00070EC8FE794E40E94440F20E030E040E8AD
:100CD0005FE30E94D70E20E030E44CE156E40E942E
:100CE000E20D0E94F20F6B017C0125E93FEB46E526
:100CF00054E30E94E20DA70196010E94E20DA701B4
:100D000096010E94E20D4B015C012FE83CEF41E4AB
:100D100059E3C701B6010E94E20D29E832ED4EE524
:100D20005AE30E94D80E9B01AC01C501B4010E9498
:100D3000D80E9B01AC0160E070E080E89FE30E9468
:100D4000440F23E333E948E853E40E94D70E6B01D4
:100D50007C01C0924004D0924104E0924204F0929F
:100D600043040E94CF0280905B0490905C04A090AA
:100D70005D04B0905E04681979098A099B09653F92
:100D8000714081059105C8F00E94CF026819790968
:100D90008A099B096C3D75408105910570F4C092EC
:100DA0003804D0923904E0923A04F0923B0469EEA0
:100DB00073E080E090E00E949D024091000150911C
:100DC00001015A834983BA01550F880B990B0E9480
:100DD000830D9B01AC01C701B6010E94E50F1816F7
:100DE0000CF0DCC08091480490914904892B09F0F3
:100DF000D5C064E670E080E090E00E949D0285EF3F
:100E000091E00E94E80264E670E080E090E00E94D9
:100E10009D02C0904004D0904104E0904204F090C4
:100E20004304A7019601C701B6010E943A10882326
:100E300019F18BE092E00E94DB0260E086E00E9404
:100E4000190260E08DE00E94190261E08CE00F90D1
:100E50000F900F900F90DF91CF911F91FF90EF9027
:100E6000DF90CF90BF90AF909F908F907F906F90CA
:100E70005F904F900C94190246015701E894B7F81F
:100E80002FEF3FEF4FE75FE7C501B4010E943A1033
:100E900081110DC02FEF3FEF4FE75FE7C501B401B0
:100EA0000E947C0D18161CF48FE092E0C4CF2FEF47
:100EB0003FEF4FE75FE4C701B6010E94E50F181648
:100EC0001CF483E192E0B7CF2FEF3FEF4FE75FECE9
:100ED000C701B6010E947C0D87FDF3CF20E030E012
:100EE000A901C701B6010E947C0D87FF09C06DE210
:100EF00081E694E00E945A01F7FAF094F7F8F09432
:100F00002AE037ED43EA5BE3C701B6010E94D80E41
:100F10004B015C010E94B60F6B017C010E94810DA8
:100F20009B01AC01C501B4010E94D70E4B015C01CD
:100F30004AE0C701B6010E94EF026EE281E694E04A
:100F40000E945A0120E030E040E251E4C501B401C2
:100F50000E94E20D4B015C010E94B60F6B01F12C67
:100F6000E12C4AE0C701B6010E94EF02C701B601B9
:100F70000E94810D9B01AC01C501B4010E94D70EF6
:100F800020E030E040E251E40E94E20D0E94B60F02
:100F900090E080E04AE00E94EF024FCF20E030E096
:100FA00048EC52ECC701B6010E947C0D87FF11C0CE
:100FB00064E670E080E090E00E949D0287E192E0AC
:100FC0000E94E80281E090E09093600480935F04C7
:100FD00034CF0E94CF02681979098A099B096132CE
:100FE0007E4481059105D0F0209138043091390478
:100FF00040913A0450913B04C701B6010E94D70EBC
:1010000020E030E040E85FE30E947C0D87FF06C0EF
:101010008091480490914904892B39F10E94CF02B4
:10102000681979098A099B0961397F4581409105D1
:1010300028F50E94CF02AB01BC018091440490913D
:101040004504A0914604B091470488519C4FAF4F8E
:10105000BF4F84179507A607B70708F16AE070E04D
:1010600080E090E00E949D0211CE64E670E080E096
:1010700090E00E949D028CE392E0A2CF8091480410
:1010800090914904892BA9F664E670E080E090E035
:101090000E949D028FE792E00E94E802CECE20E0FF
:1010A00030E04CE852E4C701B6010E947C0D87FD98
:1010B00012C069817A8164517109072E000C880B76
:1010C000990B0E94830D9B01AC01C701B6010E94E0
:1010D0007C0D87FF40C061E086E00E94190280918C
:1010E000480490914904019719F50E94CF02E091BC
:1010F0000201F09103019F01FF0F440B550B29835F
:101100003A834B835C83681979098A099B09A30197
:1011100092010E94741089819A81AB81BC81281749
:1011200039074A075B0768F561E088E00E94190209
:10113000C0923C04D0923D04E0923E04F0923F0401
:101140000E94CF0260934404709345048093460448
:101150009093470483CF20913C0430913D0440910B
:101160003E0450913F04C701B6010E94D70E2AE900
:1011700039E949E15FE30E947C0D87FDACCF60E077
:10118000ABCF0E94CF02681979098A099B09A30194
:1011900092010E94741089819A81AB81BC8182176F
:1011A0009307A407B50720F660E088E00E941902C3
:1011B00044CE60E08CE00E94190264E670E080E0BA
:1011C00090E00E949D0281EA92E00E94E80281E0A4
:1011D00090E090934904809348040E94C0051092C7
:1011E00049041092480464E670E080E090E00E94B8
:1011F0009D0283EB92E00E94E80261E08CE00C9497
:101200001902CF93DF9300D000D000D0CDB7DEB766
:1012100080E590E090930101809300010E94C00559
:1012200080915F0490916004019709F4D5C080918A
:10123000590490915A04892B41F48091570490915C
:101240005804892B11F40E94470480914C0490911A
:101250004D04019709F043C064E670E080E090E03F
:101260000E949D0287EC92E00E94E80281E694E0F1
:101270000E94180118161906CCF762ED73E08EEF84
:1012800094E00E9422050E947805CE0101960E94FA
:101290002C056CEE72E0CE0101960E94BA04882300
:1012A00009F4A3C081EF92E00E94E80210924D047D
:1012B00010924C040E94470480914C0490914D047C
:1012C0008130910541F49093600480935F048BEF2B
:1012D00092E00E94E802CE0101960E94B204809141
:1012E0005F0490916004019709F476C068EE73E0A2
:1012F00080E090E00E949D020E942F0380915F0495
:1013000090916004019709F467C00E941D0468EE83
:1013100073E080E090E00E949D020E94A60380910D
:101320005F0490916004019709F456C08AE590E04B
:1013300090930101809300010E94C00580915F0499
:1013400090916004019709F447C0809159049091ED
:101350005A04892B91F464E670E080E090E00E94EA
:101360009D028FE590E090930101809300010E941F
:10137000D90860E086E00E94190268EB7BE080E01B
:1013800090E00E949D020E942F0380915F04909143
:101390006004019709F164E670E080E090E00E944B
:1013A0009D028FE293E00E94E80268EE73E080E025
:1013B00090E00E949D0210925A04109259041092DB
:1013C00058041092570480914A0490914B0401975D
:1013D00019F4F0E0E0E0099526960FB6F894DEBF28
:1013E0000FBECDBFDF91CF910895CE0101960E942F
:1013F000B2043CCF1F920F920FB60F9211242F937D
:101400003F934F935F936F937F938F939F93AF938C
:10141000BF93EF93FF9381E694E00E943801FF9120
:10142000EF91BF91AF919F918F917F916F915F915C
:101430004F913F912F910F900FBE0F901F901895D5
:101440001F920F920FB60F9211242F938F939F9399
:10145000EF93FF93E0917104F09172048081E09129
:101460007704F091780482FD1BC0908180917A040A
:101470008F5F8F7320917B04821741F0E0917A0493
:10148000F0E0EF59FB4F958F80937A04FF91EF9135
:101490009F918F912F910F900FBE0F901F901895D5
:1014A0008081F4CF1F920F920FB60F9211242F93C9
:1014B0003F938F939F93AF93BF9380914F049091ED
:1014C0005004A0915104B091520430914E0423E095
:1014D000230F2D3758F50196A11DB11D20934E0401
:1014E00080934F0490935004A0935104B0935204FE
:1014F0008091530490915404A0915504B0915604E6
:101500000196A11DB11D8093530490935404A093A0
:101510005504B0935604BF91AF919F918F913F9125
:101520002F910F900FBE0F901F90189526E8230F54
:101530000296A11DB11DD2CFE1E6F4E01382128222
:1015400088EE93E0A0E0B0E084839583A683B78320
:101550008EE091E09183808385EC90E0958784878D
:1015600084EC90E09787868780EC90E0918B808B6D
:1015700081EC90E0938B828B82EC90E0958B848B56
:1015800086EC90E0978B868B118E128E138E148EC4
:10159000EEEFF4E01182108213821282158214821F
:1015A00050E040E062ED73E0CF010C94F704CF937C
:1015B000DF9300D000D000D0CDB7DEB7789484B5EB
:1015C000826084BD84B5816084BD85B5826085BD3F
:1015D00085B5816085BD80916E00816080936E00CD
:1015E00010928100809181008260809381008091BF
:1015F0008100816080938100809180008160809370
:1016000080008091B10084608093B1008091B0002F
:1016100081608093B00080917A00846080937A002A
:1016200080917A00826080937A0080917A00816054
:1016300080937A0080917A00806880937A0010927B
:10164000C10061E086E00E94470261E088E00E94FC
:10165000470261E089E00E94470261E087E00E9462
:10166000470261E08AE00E94470261E08BE00E944D
:10167000470261E08DE00E94470261E08CE00E9439
:10168000470260E082E00E94470260E085E00E943D
:10169000470260E085E10E94470260E084E00E942A
:1016A000470260E083E00E94470260E089E00E9418
:1016B000190260E088E00E94190260E086E00E9462
:1016C000190260E087E00E94190260E08AE00E944F
:1016D000190260E08BE00E94190260E08DE00E9438
:1016E000190260E08CE00E941902E0917104F0910F
:1016F000720482E08083E0916D04F0916E041082A8
:10170000E0916F04F09170048FEC80831092790463
:10171000E0917504F091760486E08083E091730493
:10172000F0917404808180618083E0917304F09172
:101730007404808188608083E0917304F091740464
:10174000808180688083E0917304F09174048081CB
:101750008F7D808364E670E080E090E00E949D02CF
:101760008AE393E00E94E80201E010E040E5242EC5
:10177000312C5FE0E52EF12C64E6462E512C8CE3F3
:10178000C82ED12C99E1A92EB12C24E1822E912CC6
:1017900030E0632E30E0732E61E08CE00E9419028D
:1017A00080915F0490916004019709F04CC00E9401
:1017B000CF0260935B0470935C0480935D0490930C
:1017C0005E0464E670E080E090E00E949D028EE49A
:1017D00093E00E94E80264E670E080E090E00E94FE
:1017E0009D0283E693E00E94E80260E08CE00E94A4
:1017F000190261E08DE00E94190268EE73E080E05A
:1018000090E00E949D0260E08DE00E94190268EE67
:1018100073E080E090E00E949D020E94CF02209140
:101820005B0430915C0440915D0450915E04621B46
:10183000730B840B950B6033754781059105C9F6D1
:10184000F0E0E0E0099581E694E00E9418011816A6
:1018500019060CF01AC162ED73E08EEF94E00E945D
:1018600022050E947805CE0101960E942C056EE7A4
:1018700073E0CE0101960E94BA04882371F064E6F9
:1018800070E080E090E00E949D0283E893E00E9477
:10189000E802F0920301E09202016EE873E0CE01EB
:1018A00001960E94BA04882371F064E670E080E03B
:1018B00090E00E949D0283E993E00E94E8029092EA
:1018C0000301809202016DE973E0CE0101960E944E
:1018D000BA04882371F064E670E080E090E00E9432
:1018E0009D0282EA93E00E94E802B0920301A09276
:1018F000020169EA73E0CE0101960E94BA048823CE
:1019000071F064E670E080E090E00E949D028EEA53
:1019100093E00E94E802D0920301C092020169EBB9
:1019200073E0CE0101960E94BA04882361F064E658
:1019300070E080E090E00E949D028EEB93E00E94B8
:10194000E8020E94010963ED73E0CE0101960E9456
:10195000BA04882381F064E670E080E090E00E94A1
:101960009D0288ED93E00E94E80210935A040093D0
:1019700059040E94010960EE73E0CE0101960E94B5
:10198000BA048823B1F064E670E080E090E00E9441
:101990009D0285EE93E00E94E8028CE090E0909337
:1019A00003018093020110935804009357040E948E
:1019B00001096BEE73E0CE0101960E94BA04811119
:1019C0000E94470460EF73E0CE0101960E94BA04C2
:1019D000882331F0F0920301E09202010E94D908BD
:1019E00065EF73E0CE0101960E94BA0481110E9456
:1019F000A6036AEF73E0CE0101960E94BA0481113A
:101A00000E942F036FEF73E0CE0101960E94BA048B
:101A1000882331F030920101209200010E94C0051C
:101A200064E074E0CE0101960E94BA0481110E9424
:101A30001D0469E074E0CE0101960E94BA04882377
:101A400001F164E670E080E090E00E949D028EE08B
:101A500094E00E94E80210935A04009359040E94F3
:101A6000010910935804009357040E94010964E689
:101A700070E080E090E00E949D0287E194E00E9487
:101A8000E802CE0101960E94B20485E00E94F001B6
:101A90000197E1F4509201014092000189E294E043
:101AA0000E94E80264EF71E080E090E00E949D02F5
:101AB0000E94C00560E27EE480E090E00E949D020A
:101AC00080915F04909160040197F9F66AE070E0FC
:101AD00080E090E00E949D026114710409F45CCEE4
:101AE0000E942401882309F44ACE0E94000047CEB8
:101AF0008EEF94E00C94B2040E94BE0D08F481E0D5
:101B00000895E89409C097FB3EF4909580957095F0
:101B100061957F4F8F4F9F4F9923A9F0F92F96E939
:101B2000BB279395F695879577956795B795F111AE
:101B3000F8CFFAF4BB0F11F460FF1BC06F5F7F4F4B
:101B40008F4F9F4F16C0882311F096E911C077235D
:101B500021F09EE8872F762F05C0662371F096E866
:101B6000862F70E060E02AF09A95660F771F881F35
:101B7000DAF7880F9695879597F90895990F0008D9
:101B8000550FAA0BE0E8FEEF16161706E807F9074F
:101B9000C0F012161306E407F50798F0621B730BEA
:101BA000840B950B39F40A2661F0232B242B252B6B
:101BB00021F408950A2609F4A140A6958FEF811D0E
:101BC000811D08950E94F50D0C94660E0E94580E1A
:101BD00038F00E945F0E20F0952311F00C944F0E08
:101BE0000C94550E11240C949A0E0E94770E70F3EB
:101BF000959FC1F3950F50E0551F629FF001729FB2
:101C0000BB27F00DB11D639FAA27F00DB11DAA1FC0
:101C1000649F6627B00DA11D661F829F2227B00D0D
:101C2000A11D621F739FB00DA11D621F839FA00D98
:101C3000611D221F749F3327A00D611D231F849FE8
:101C4000600D211D822F762F6A2F11249F5750403F
:101C50009AF0F1F088234AF0EE0FFF1FBB1F661FBA
:101C6000771F881F91505040A9F79E3F510580F083
:101C70000C944F0E0C949A0E5F3FE4F3983ED4F30D
:101C8000869577956795B795F795E7959F5FC1F727
:101C9000FE2B880F911D9695879597F9089597F9D2
:101CA0009F6780E870E060E008959FEF80EC089502
:101CB00000240A941616170618060906089500242B
:101CC0000A9412161306140605060895092E0394A5
:101CD000000C11F4882352F0BB0F40F4BF2B11F419
:101CE00060FF04C06F5F7F4F8F4F9F4F089557FD78
:101CF0009058440F551F59F05F3F71F04795880F7A
:101D000097FB991F61F09F3F79F087950895121610
:101D100013061406551FF2CF4695F1DF08C01616BC
:101D200017061806991FF1CF86957105610508946D
:101D30000895E894BB2766277727CB0197F9089584
:101D40002F923F924F925F926F927F928F929F92CB
:101D5000AF92BF92CF92DF92EF92FF920F931F93B9
:101D6000CF93DF93CDB7DEB7CA1BDB0B0FB6F8946A
:101D7000DEBF0FBECDBF09942A88398848885F84AA
:101D80006E847D848C849B84AA84B984C884DF801B
:101D9000EE80FD800C811B81AA81B981CE0FD11DFF
:101DA0000FB6F894DEBF0FBECDBFED0108955058B9
:101DB000BB27AA270E94EF0E0C94660E0E94580EB5
:101DC00038F00E945F0E20F039F49F3F19F426F49A
:101DD0000C94550E0EF4E095E7FB0C944F0EE92F92
:101DE0000E94770E58F3BA176207730784079507A6
:101DF00020F079F4A6F50C94990E0EF4E0950B2ED4
:101E0000BA2FA02D0B01B90190010C01CA01A0014C
:101E10001124FF27591B99F0593F50F4503E68F1A7
:101E20001A16F040A22F232F342F4427585FF3CFE8
:101E3000469537952795A795F0405395C9F77EF4B9
:101E40001F16BA0B620B730B840BBAF09150A1F002
:101E5000FF0FBB1F661F771F881FC2F70EC0BA0F88
:101E6000621F731F841F48F4879577956795B79510
:101E7000F7959E3F08F0B0CF9395880F08F099270B
:101E8000EE0F9795879508950E94580F0C94660E53
:101E90000E945F0E58F00E94580E40F029F45F3FF8
:101EA00029F00C944F0E51110C949A0E0C94550E6F
:101EB0000E94770E68F39923B1F3552391F3951B94
:101EC000550BBB27AA2762177307840738F09F5F5B
:101ED0005F4F220F331F441FAA1FA9F335D00E2EC8
:101EE0003AF0E0E832D091505040E695001CCAF735
:101EF0002BD0FE2F29D0660F771F881FBB1F2617F8
:101F000037074807AB07B0E809F0BB0B802DBF01CE
:101F1000FF2793585F4F3AF09E3F510578F00C949D
:101F20004F0E0C949A0E5F3FE4F3983ED4F38695DF
:101F300077956795B795F7959F5FC9F7880F911DBE
:101F40009695879597F90895E1E0660F771F881FAA
:101F5000BB1F621773078407BA0720F0621B730B5D
:101F6000840BBA0BEE1F88F7E09508950E947F0E50
:101F700088F09F5798F0B92F9927B751B0F0E1F04A
:101F8000660F771F881F991F1AF0BA95C9F714C0FA
:101F9000B13091F00E94990EB1E008950C94990E21
:101FA000672F782F8827B85F39F0B93FCCF3869533
:101FB00077956795B395D9F73EF490958095709590
:101FC00061957F4F8F4F9F4F08950E94BE0D08F47B
:101FD0008FEF089516F00C943F100C94550E6894F2
:101FE0000C944F0E0E947F0EA8F39923C1F3AEF319
:101FF000DF93CF931F930F93FF92C92FDD27882381
:102000002AF02197660F771F881FDAF720E030E06B
:1020100040E85FEB9FE3883920F0803E38F021965E
:102020008F770E94D80EE8E6F0E004C00E94D80E38
:10203000E5E9F0E00E944D108B01BE01EC01FB2EA2
:102040006F5771097595771F880B990B0E94830D47
:1020500028E132E741E35FE30E94F50DAF2D9801DF
:10206000AE01FF900F911F91CF91DF910E94EF0E73
:102070000C94660E0E94BE0D880B990B08959F3F2D
:1020800031F0915020F4879577956795B795880F33
:10209000911D9695879597F90895DF93CF931F9398
:1020A0000F93FF92EF92DF927B018C01689406C040
:1020B000DA2EEF010E94F50DFE01E894A59125911D
:1020C000359145915591A6F3EF010E94EF0EFE0167
:1020D0009701A801DA9469F7DF90EF90FF900F91D4
:1020E0001F91CF91DF910895A1E21A2EAA1BBB1B6D
:1020F000FD010DC0AA1FBB1FEE1FFF1FA217B307D4
:10210000E407F50720F0A21BB30BE40BF50B661FE9
:10211000771F881F991F1A9469F7609570958095AD
:1021200090959B01AC01BD01CF010895EE0FFF1FFB
:102130000590F491E02D09940F931F93CF93DF93B3
:102140008230910510F482E090E0E0910605F09174
:10215000070530E020E0B0E0A0E0309799F42115C9
:10216000310509F44AC0281B390B24303105D8F554
:102170008A819B816115710589F1FB0193838283BB
:10218000FE0111C040815181028113814817590716
:10219000E0F04817590799F4109761F012960C93E4
:1021A000129713961C933296CF01DF91CF911F9116
:1021B0000F9108950093060510930705F4CF21159C
:1021C000310551F04217530738F0A901DB019A019C
:1021D000BD01DF01F801C1CFEF01F9CF90930705F1
:1021E00080930605CDCFFE01E20FF31F81939193FB
:1021F0002250310939832883D7CF209104053091AB
:102200000505232B41F420910601309107013093FD
:102210000505209304052091040130910501211545
:10222000310541F42DB73EB74091080150910901A5
:10223000241B350BE0910405F0910505E217F30727
:10224000A0F42E1B3F0B2817390778F0AC014E5F26
:102250005F4F2417350748F04E0F5F1F5093050559
:1022600040930405819391939FCFF0E0E0E09CCFF1
:10227000CF93DF930097E9F0FC013297138212822B
:10228000A0910605B0910705ED0130E020E0109720
:10229000A1F420813181820F931F20910405309198
:1022A00005052817390709F061C0F0930505E0938B
:1022B0000405DF91CF910895EA01CE17DF07E8F515
:1022C0004A815B819E0141155105B1F7E901FB830C
:1022D000EA8349915991C40FD51FEC17FD0761F4AA
:1022E000808191810296840F951FE90199838883EB
:1022F000828193819B838A83F0E0E0E012968D9146
:102300009C9113970097B9F52D913C911197CD01B0
:102310000296820F931F209104053091050528171E
:10232000390739F6309751F51092070510920605D6
:10233000B0930505A0930405BCCFD383C28340812D
:102340005181840F951FC817D90761F44E5F5F4F05
:1023500088819981480F591F518340838A819B81CD
:10236000938382832115310509F0B0CFF0930705DF
:10237000E09306059ECFFD01DC01C0CF13821282DF
:10238000D7CFB0E0A0E0E7ECF1E10C94A20E8C0115
:10239000009751F4CB010E949C108C01C801CDB76D
:1023A000DEB7E0E10C94BE0EFC01E60FF71F9C01C6
:1023B00022503109E217F30708F49DC0D901CD91ED
:1023C000DC911197C617D70798F0C530D10530F3C7
:1023D000CE0104978617970708F3C61BD70B2297E1
:1023E000C193D1936D937C93CF010E943811D6CFC6
:1023F0005B01AC1ABD0A4C018C0E9D1EA091060516
:10240000B0910705512C412CF12CE12C109731F59E
:1024100080910405909105058815990509F05CC027
:102420004616570608F058C08091040190910501A6
:10243000009741F48DB79EB7409108015091090172
:10244000841B950BE817F90708F055C0F0930505B4
:10245000E0930405F90171836083A0CF8D919C9175
:10246000119712966C90129713967C901397A8155B
:10247000B90559F56C0142E0C40ED11CCA14DB0445
:1024800020F1AC014A195B09DA011296159780F028
:102490006282738251834083D9016D937C93E114EE
:1024A000F10471F0D7011396FC93EE93129776CF57
:1024B00022968C0F9D1FF90191838083F301EFCF4A
:1024C000F0930705E093060569CF4816590608F40E
:1024D0002C017D01D3019ACFCB010E949C107C017D
:1024E000009749F0AE01B8010E947E12C8010E9417
:1024F0003811870153CF10E000E050CFFB01DC0121
:1025000002C001900D9241505040D8F70895FB0150
:10251000DC018D91019080190110D9F3990B089578
:10252000FB01DC0101900D920020E1F7089510E01D
:10253000CFE8D0E004C0FE010E9496102196C03979
:10254000D107C9F7F894FFCF46000F000000080537
:102550008000000000005A01BA00E700A70118013E
:10256000F6000A01756E5072657373696E672E2EE0
:102570002E0A00556E507265737365640A00752DDE
:10258000656E64206F6620756E5072657373696E38
:1025900067206E6F742064657465637465640A00F7
:1025A0007072657373696E672E2E2E0A00702D652A
:1025B0006E64206F66207072657373696E67206E3B
:1025C0006F742064657465637465640A0064726F77
:1025D0007070696E672E2E2E0A0044726F707065DF
:1025E000640A006772696E64696E672E2E2E0A0097
:1025F0004772696E64696E6720446F6E650A0057A2
:1026000061726E696E672C206772696E64696E67AD
:1026100020746F6F6B20746F6F206C6F6E67210A70
:10262000004F7574206F6620436F666665653F0ACC
:102630000048656174696E6720746F20007265617F
:102640006368656420646573697265642074656D90
:10265000700A006E616E00696E66006F76660075C6
:102660002D546865726D6F636F75706C653A207577
:102670006E706C7567676564206F72206661696C47
:1026800065640A00702D546865726D6F636F7570B4
:102690006C653A206E6F7420646574656374696E4E
:1026A000672068656174696E672C20706F73697448
:1026B000696F6E696E67206F722072656C61792038
:1026C0006661756C740A00682D74616B696E6720B1
:1026D000746F6F206C6F6E672C20636F6E74696E01
:1026E00075696E672E2E2E0A0070756D70696E67A3
:1026F0002057617465722E2E2E0A0050756D706918
:102700006E6720776174657220646F6E650A00726F
:102710006566696C6C20636F6666656520616E64D2
:102720002073656E6420636F6E7420636F6D6D61DE
:102730006E640A00636F6E7400526566696C6C6546
:10274000640A00672D6661696C7572653A2073656D
:10275000636F6E64206772696E64696E672066617C
:10276000696C7572652C20636865636B206772699C
:102770006E646572210A00436F6D706C657465212B
:102780000A0041726475696E6F2072756E6E696EB3
:1027900067203A290A004572726F722068617320BF
:1027A0006F636375727265642E0A00436865636BBC
:1027B000206D616368696E6520616E642072657367
:1027C000746172740A00726973740052697374726E
:1027D0006574746F0A00657370720045737072657A
:1027E00073736F0A006C6F6E67004C756E676F0ACB
:1027F00000616D657200416D65726963616E6F0A9B
:10280000006D616B65004D616B696E6720736F6D64
:102810006520636F66666565210A006472797200DF
:1028200044727952756E0A006E6F636F004E6F438B
:102830006F0A006772696E0070756D700070726566
:102840007300756E707200686561740064726F70F9
:1028500000636C656100732D636C65616E0A0053E3
:102860002D636C65616E696E6720646F6E652E0AFC
:10287000005661706F722068656174696E670A0046
:107E0000112484B714BE81FFF0D085E080938100F7
:107E100082E08093C00088E18093C10086E0809377
:107E2000C20080E18093C4008EE0C9D0259A86E02C
:107E300020E33CEF91E0309385002093840096BBD3
:107E4000B09BFECF1D9AA8958150A9F7CC24DD24C4
:107E500088248394B5E0AB2EA1E19A2EF3E0BF2EE7
:107E6000A2D0813461F49FD0082FAFD0023811F036
:107E7000013811F484E001C083E08DD089C08234E0
:107E800011F484E103C0853419F485E0A6D080C0E4
:107E9000853579F488D0E82EFF2485D0082F10E0AE
:107EA000102F00270E291F29000F111F8ED06801E7
:107EB0006FC0863521F484E090D080E0DECF843638
:107EC00009F040C070D06FD0082F6DD080E0C81688
:107ED00080E7D80618F4F601B7BEE895C0E0D1E017
:107EE00062D089930C17E1F7F0E0CF16F0E7DF06D8
:107EF00018F0F601B7BEE89568D007B600FCFDCFD4
:107F0000A601A0E0B1E02C9130E011968C91119780
:107F100090E0982F8827822B932B1296FA010C0160
:107F200087BEE89511244E5F5F4FF1E0A038BF0790
:107F300051F7F601A7BEE89507B600FCFDCF97BE46
:107F4000E89526C08437B1F42ED02DD0F82E2BD052
:107F50003CD0F601EF2C8F010F5F1F4F84911BD097
:107F6000EA94F801C1F70894C11CD11CFA94CF0C13
:107F7000D11C0EC0853739F428D08EE10CD085E9AC
:107F80000AD08FE07ACF813511F488E018D01DD067
:107F900080E101D065CF982F8091C00085FFFCCF94
:107FA0009093C60008958091C00087FFFCCF809118
:107FB000C00084FD01C0A8958091C6000895E0E648
:107FC000F0E098E1908380830895EDDF803219F02E
:107FD00088E0F5DFFFCF84E1DECF1F93182FE3DFCA
:107FE0001150E9F7F2DF1F91089580E0E8DFEE27F6
:047FF000FF270994CA
:027FFE00040479
:00000001FF
